:0300000002238A4E
:10238A0043AF01787FE4F6D8FD75A000758121027C
:02239A0023D747
:10000E0090E000EFF0781ED8FE2290E001EFF0783D
:04001E001ED8FE22C8
:022DA900010126
:10299200E490014DF0A312041F0000000078527C65
:1029A200017D017BFF7A2D79A97E007F021200F65C
:1029B200122C86122D72122D5C122CB6122C1612AB
:0E29C20027E9EF600612287E122A700212A486
:102A3C0053797374656D204D656E752F4261636BB0
:102A4C00003E2000373839483435364B3132334D5F
:102A5C004E302E526D2B2D21444342413C4F3E2093
:042A6C0020202045C1
:081991004101ED004101EB00F2
:101FF5009001901203FBE47B0AFAF9F82290017430
:1020050012040712026B90017812041390015E12FC
:1020150003FB900178120407D30203BE90017812E6
:10202500041390015A1203FB900178120407C302AE
:1020350003BE9001781203FB900174221202869070
:1020450001900204139001740203FBD3900198E000
:102055006480948022C3900189E0FF90019AE09FFB
:102065002212290B90018C02041390018C1203FBA0
:10207500EC4D4E4F2290016CE0FF90016BE022FF8A
:10208500900189E0FEC3EF9E229001801203FB9030
:1020950001902290016DE0FF900166120453EF025A
:1020A5000184900162E0FF900164E02F2290019885
:1020B500E004F0229001780204139001CC0204534D
:0C2D5C00E4F590E59054069001ECF022A4
:1026F500E590540170037F2122E4FFEF3333335417
:10270500F8FEE5B054C74E4403F5B0E590F45478AF
:10271500131313541FFE602CE4FDEE602730E01DFB
:1027250075F004EFA42DF582E435F0F583E58224F8
:1027350050F582E583342AF583E493FF22EEC31333
:0B274500FE0D80D60FEFB407B27F003E
:012750002266
:062D84009001EBEFF022CC
:10253300E49001A0F09001EFE06003120F799001A5
:10254300EBE0FF600A90019FF0E49001EBF02212B0
:1025530026F590019FEFF060369001EDE0FF9001CA
:102563009FE06F7015122D20EF602F7F647E0012A5
:102573002D7B90019FE0A3F080207FF47E01122D3C
:102583007B90019FE09001EDF09001A0F0800B1291
:102593002D20EF6005E49001EDF09001A0E0B44F31
:0925A30003122D309001A0E0FFAD
:0125AC00220C
:102D0000EF6009E5B054FB4403F5B02243B007225D
:10294F00EF24FE601914601A14601B1460261460C3
:10295F00272405702D7F48122D687F7A80217F25CF
:10296F00801D7F5680197F64122D687F42122D685B
:10297F007F6D800B7FDF80077FE4122D687F7312DE
:03298F002D68228E
:06086F0090017C1204134D
:1008750090018C12041F00000000E4900198F0A381
:1008850004F0E490019BF0020C0F900199E07003D5
:10089500020946122D9F900188E0FF90019DF0907E
:1008A500019BE0600E900198E0700890019DE0606A
:1008B5000214F01220851475F00384A3E02480C38C
:1008C50095F0FF122ACD122D8A90018AE0FEEFC322
:1008D5009E50077F20122D6880EC90018C1203FB3F
:1008E5009001A012041390019DE09001A4F09001E5
:1008F50098E09001A5F090018AE0FF121EDF9001BB
:100905009BE06015900198E0700F122D8A90019C74
:10091500EFF07F2E122D688009122D8AEF149001B9
:100925009CF07F20122D6890018BE0FF12294F7FEC
:1009350020122D6890019CE02480FF122ACD122DF3
:1009450095122533900199EFF012047C0A67210A6C
:10095500C72E098E30098E31098E32098E33098EE4
:1009650034098E35098E36098E37098E38098E3948
:100975000C17450AEE480B024B0B714D0AD04E0B76
:10098500EC520C176D0000088F7F007E2D7D317CA9
:100995000190018C12201A400302088F7F007ED33C
:1009A5007DCE7CFE90018C122030500302088F9082
:1009B5000198E064809486400302088FE47F0AFE74
:1009C500FDFC90018C12040712204190019EE090DD
:1009D5000190B40113120407900199E024D0FFE4BB
:1009E500FCFDFE12026B80171203FBEFC0E09001C5
:1009F50099E024D0FBE4FAF9F8D0E0FF120278126E
:100A050020449001901203FB90019412041390016D
:100A15009BE0FF900198E02F90019AF012205A5028
:100A250017900194121FF812028690019412041374
:100A350090019AE004F080E4900198E0FB70089042
:100A4500019BE07002800F90019BE07006EB700344
:100A550002088F1220B29001901203FB1220690246
:100A6500088F900198E090019AF0D312205B401115
:100A750090018C121FF812206690019AE014F08004
:100A8500E912205A501490018C121FF81202861296
:100A9500206990019AE004F080E79001801203FB41
:100AA50090018C1220305003020B419001841203F7
:100AB500FB90018C12201A4003020B5290018C020C
:100AC5000C1A90019B7401F002088F90018C12039F
:100AD500FB1203B012206912206F700302088F9079
:100AE500019EE0F404F002088F90018BE0FF6401A1
:100AF5006008EF6403600302088F020BDF90018B2F
:100B0500E064017059900198E024FD122084900161
:100B150098F01220504011121FF512290B12204493
:100B2500900198E014F080EAC3122051502A121F58
:100B3500F512204112208E122030500690018002BD
:100B45000C1A90018412209112201A4006900184FB
:100B5500020C1A1220B280D0900190020C1A90015A
:100B65008BE06404600302088F020BDF90018BE0C9
:100B75006401705B900198E024FA1220849001983A
:100B8500F01220504011121FF512290B122044902B
:100B95000198E014F080EA900198E0C364809480A5
:100BA5005028121FF512204112208E1220305005B8
:100BB500900180806090018412209112201A4005D6
:100BC50090018480501220B280CD90019080469093
:100BD500018BE06405600302088F7F21122D84E4F8
:100BE500900199F002088F90018C121FF81220666F
:100BF500900198E0600214F0900198E07004900173
:100C05009BF012206F600302088F90019E04F00292
:080C1500088F90017C1203FB23
:010C1D0022B4
:0604BB009001561204132B
:1004C1009001697401F090016612045312011C90AD
:1004D100016DF0E4A3F0A3F0A312041F00000001DA
:1004E10090015612203A12041390015E12203A1222
:1004F100201A400990015E12203A12041390015A09
:1005010012203A122030500990015A12203A120456
:100511001390016B7401F090016D12207DC39F5007
:1005210017900170121FF8120286900170120413C5
:1005310090016BE004F080DF900169E07003020636
:100541009A12204AEC3390017450081203FB1203F3
:10055100B080031203FB1220B990016DE0FF9001FE
:100561006CF0900163E004FED39F400790016CEEB4
:10057100F0800890016DE090016CF01220A71490BA
:10058100016AF0A37401F0E490016FF0122D9F90C5
:10059100016AE004547F2480FF122ACD7F20122DAE
:1005A10068900165E0FF12294F9001781220727066
:1005B1000712207AD39F506812084D121FFB900139
:1005C100781203FB12290BEB2430FF122D689001E6
:1005D10078121FF812290B1220B990016312207DA5
:1005E1006F700A12084D7F2E122D68802A900163C8
:1005F10012207DFED39F401FEE9F75F00384E5F02E
:10060100701512085E7F20122D6812207AC39F5048
:100611000690016FE004F090016BE004F00205AA7E
:1006210012204AEC33500812085E7F2D122D68907B
:100631000163E0FF900162E0C39F1475F00384FF42
:10064100900164E0547F2480C39FFF122ACD122DB4
:100651008A90016AE0FEEFD39E50077F20122D6839
:1006610080EC1220A7FF90016DE0FEC3EF9EFF908A
:10067100016FE0FDC3EF9DFF900163E0FDEED39DAF
:100681004007ED60047E0180027E00C3EF9E547F2F
:100691002480FF122ACD122D95122533900169EF86
:1006A100F012047C07622B07752D07922E079230FA
:1006B1000792310792320792330792340792350736
:1006C100923607923707923807923906EB3C072991
:1006D1003E07E74107E74207E74307E74407F145DC
:1006E10007474E07E76D000007F690015A1203FB1A
:1006F100EC3350047F0180027F00900163E06004CD
:100701007E0180027E00900162E0C39EC39FFF9044
:10071100016DE0C39F4003020832E004F0900170D4
:10072100121FF8120286801890016DE0D3940150D7
:1007310003020832E014F0900170121FF812290B25
:1007410090017002078C12204A1203B0122021502E
:1007510003020832122011400302083212203780AE
:100761002A9001701203FB12200240030208321288
:100771002037801790017012040712204A12027864
:1007810012202150030208321220371204130208EA
:1007910032900169E0FF122D8412209890015A12C3
:1007A10003FB90018012041390015E1203FB900180
:1007B10084120413900162E0900188F0900163E0DB
:1007C100900189F0900164E090018AF0900165E068
:1007D10090018BF012204A12086F900174120413D9
:1007E100122BD3020849900169E0FF122D84800089
:1007F10090016E8039122D10EE3395E0FDFC122030
:10080100B99001781220726028122BD390017012D6
:1008110003FB900178120407120286122002501184
:10082100122027400C122037120413900169740121
:10083100F012204A900156122030700990016EE0AA
:0B084100700302053912209812204AB3
:10084C002290016AE0FF14F0EF547F2480FF122AFB
:10085C00CD2290016AE0FF14F0EF547F2480FF1248
:03086C002ACD2270
:0B1CA1009001C61204739001C5EFF023
:101CAC009001CFF0A37401F01220BF9001D2120466
:101CBC0073122D9F7F01122ACD7BFF7A2A793CE487
:101CCC00FF122A9F9001C61204537F40122A9F7B59
:101CDC00FF7A2A794D7F14122A9F9001C91204535E
:101CEC007F54122A9F9001D2E475F00112045C1209
:101CFC00011C70F11220BFCFE9CF9001D212045316
:101D0C00C3E99FFFC374699FFF1220BF122A9F90E3
:101D1C0001D0E06040122D9F9001CFE06005900152
:101D2C00C980039001CC1204537F16122A9F122DE6
:101D3C008A9001D1EFF0122D8AEFC3942850077FBF
:101D4C0020122D6880F09001D1E0547F2480FF1286
:101D5C002ACD122D951225339001D0EFF012047C70
:101D6C001D9E211D852B1D852D1D91411D96441DEC
:101D7C00A4521DA46D00001DAA9001CFE0FFC374F6
:101D8C00019FF0808A9001CF8029E49001CFF0026E
:101D9C001D1B9001CFE0FF229001C5E0FF22122D08
:101DAC0010EF4E7003021D1B122BD39001CFE06479
:091DBC0001F0A37401F0021D1BEB
:101999004101DD004101DE004201D500004201D7CD
:1019A90000004401DF020003014401D901030002E0
:10223C009001D5E0FDA3E09001C3CDF0A3EDF0E556
:10224C0090C3135403FE9001DEE0C3940A50047F44
:10225C000280027F0174D92EF582E43401F583E00B
:10226C00FD9001DDE0F9ED697020EFFDC39001D622
:10227C00E09DF09001D5E09400F0C39001D8E09D72
:10228C00F09001D7E09400F0802274DF2EF582E408
:10229C003401F583E0697014EFFD9001D5E48DF005
:1022AC001202559001D7E48DF01202559001D5A37E
:1022BC00E054FCFD9001C3A3E054FC6D6007E49076
:1022CC0001DEF0800C9001DEE0C394FF5003E004CB
:0622DC00F09001DDEEF0C0
:0122E20022D9
:102CDD009001D5E0FEA3E07802CEC313CE13D8F950
:022CED00FF22C4
:102C5300EF7802C333CE33CED8F9FF9001D5EEF02F
:0A2C6300A3EFF0A3EEF0A3EFF022C0
:102BD300E49001D5F0A3F09001D8E02404FF900124
:102BE300D7E03400FE7C007D0412021FECF0A3ED5D
:022BF300F022CE
:102D10009001D7E0FEA3E0FF7C007D0412021F2299
:102AF7009001B2E0FF04F074A62FF582E43401F5EB
:102B07008322FF9001B2E0FEEF6480F8EE648098C4
:082B170022F09001A00203FB73
:042D90007F1EDFFEC5
:012D9400221C
:062D8A009001F0E0FF22C1
:052D95007F0F022ACDB2
:052D9A007F0E022ACDAE
:052D9F007F0C022ACDAB
:052ACD009001B5EFF0DF
:102AD20012000E9001B5E0FF30E706547F9001F03E
:102AE200F09001B5E0C39404500AE4FE122D900E5A
:042AF200EEB418F82E
:012AF60022BD
:0A2D68001200189001F0E004F022C0
:102A9F0090016F120473EF547F2480FF122ACD90A0
:102AAF00016F12045312011C601390016FE475F053
:0E2ABF000112045C12011CFF122D6880E2223D
:051EDF0090019FEFF0EF
:101EE400E49001B2F0A3F0A3122B18EC335011903C
:101EF40001B37401122B181203B09001A012041341
:101F0400122B19EC4D4E4F604AE47B0AFAF9F81291
:101F14002B1912290BEB2430FF9001B2E0FE04F0E0
:101F240074A62E122B01EF122B18E47B0AFAF9F88F
:101F340012290B9001A01204139001A5E0FF900157
:101F4400B2E06F70BB122AFA742EF09001B47401DF
:101F5400F080AD9001B2E0700C9001A67430F09066
:101F640001B2E004F09001A5E0602B04D3122B0928
:101F740050249001A5E0C3122B095008122AFA74C8
:101F840030F080EE9001B4E07006122AF7742EF05F
:101F9400122AF77430F090019FE0547F2480FF12DE
:101FA4002ACD9001B3E060069001A4E014F0900102
:101FB400B2E014F09001A4E014FFF09001B2E0FE4E
:101FC400C3122B0F50077F20122D6880E79001B3B6
:101FD400E060057F2D122D689001B2E024A6122B3B
:101FE40001E0FF122D689001B2E0FF14F0EF70E8F9
:011FF40022CA
:102CB6007F38122ACD7F01122ACD7F0F122ACD7FAF
:042CC60001022C6D6E
:092D7200438780759870D2AC22F1
:102C8600758921758CFC758A6BD28CD2A9D2AF75E9
:082C96008DFD758BFDD28E222D
:102CCA009001E3EEF0A3EFF09001E3E07002A3E0DD
:032CDA0070F6226F
:102C9E009001E3E07002A3E060037F00229001E365
:082CAE00EEF0A3EFF07F01221C
:092D7B009001E7EEF0A3EFF02255
:102D20009001E7E07002A3E060037F00227F0122B0
:102C35009001E9EEF0A3EFF09001E9E07002A3E066
:0E2C450060069001EFE060F09001EFE0FF22EA
:0700030074FFF5F002025545
:03000B0002241CB0
:10241C00C0E0C0F0C083C082C0D0E8C0E0E9C0E03A
:10242C00EAC0E0EBC0E0ECC0E0EDC0E0EEC0E0EFF5
:10243C00C0E0758CFC758A6B9001E3E07002A3E040
:10244C0060069001E31200039001E5E07002A3E046
:10245C0060069001E51200039001E7E07002A3E032
:10246C0060069001E71200039001E9E07002A3E01E
:10247C0060069001E912000312223CD0E0FFD0E08C
:10248C00FED0E0FDD0E0FCD0E0FBD0E0FAD0E0F9EB
:0E249C00D0E0F8D0D0D082D083D0F0D0E032A3
:03002300022B6A43
:102B6A00C0E0C083C082309808C2989001EF740117
:102B7A00F0309908C2999001EE7401F0D082D083A6
:032B8A00D0E03266
:1019B900604400740000000003AA0000000024A68F
:1019C900000000016E810000000E510A0000008F26
:1019D9002A6300000597A7E0000037EC8EC20002D9
:1019E9002F3D93980015D867C3ED00DA740DA74110
:1019F9000888888888880000410073806064000F27
:101A09000FFF0FD00FA10F730F460F190EED0EC167
:101A19000E960E6B0E410E170DEE0DC50D9D0D7533
:101A29000D4E0D270D000CDA0CB40C8F0C6A0C4608
:101A39000C220BFE0BDB0BB80B960B740B530B3103
:101A49000B110AF00AD00AB00A910A720A530A3530
:101A59000A1709FA09DC09C009A30987096B094FA3
:041A6900093409191A
:1025AD00CD122D409001AE1203FB78081203E79077
:1025BD0001AE1204139001AE0203FBED25E0240FD2
:1025CD00F582E43400F583E0FFA3E09001AECFF097
:1025DD00A3EFF0229001AF0203FB9001AF120413A1
:1025ED009001AF0203FB74B32DF58274013CF583AA
:1025FD002274B32FF58274013EF583229DFDE49C78
:10260D00FCC364809480222DFD74FF3CFC22D3ED2D
:08261D009431EC6480948022EA
:10287E00900154E4F0A37404F0A37411F07B017A78
:10288E00007974A3120473900156E0FF14F0EF6008
:10289E0025A3120453900154E0FCA3E0FD122BB0CB
:1028AE00900158E475F004120255900154E475F04D
:0628BE000412025580D156
:0128C40022F1
:102C160090A000740BF0E4FFFE0FBF00010EBE0390
:0F2C2600F8BFE7F590A0007409F0E4FF022BF56A
:0E2D4000CEEDCEEFFD74808D82F583EEF02295
:102A07009001BEEFF0A31204739001C2E0FF14F02F
:102A1700EF60219001BFE475F00112045C12011C04
:102A2700FF9001BEE0FE04F0EEFD74808D82F58319
:052A3700EFF080D52244
:102BF500CDEFCDEF9000736006E04401F08004E076
:102C050054FEF0900073E090C000F0CFEDCF022DA0
:012C150000BE
:102D3000900073E020E0047F0180027F00022BF509
:102CEF00900073E05481FEEF547E4EF090C000F0E0
:012CFF0022B2
:102C6D00EF9000736006E04480F08004E0547FF044
:092C7D00900073E090C000F02209
:051B56009001AEEFF06C
:101B5B00E49001B9F09001B9E0FFC39406501474FE
:101B6B00B32FF582E43401F583E4F09001B9E0047E
:101B7B00F080E29001BA7411F01225E1EC4D4E4F5A
:101B8B007003021C8D9001BAE02406F0E0C3943C74
:101B9B0040141225E19001BBEFF09001AF12041F2E
:101BAB00000000008023E47B0AFAF9F81225E11209
:101BBB00290B9001BBEBF01225E1E47B0AFAF9F853
:101BCB0012290B9001AF1204139001BBE060AAE441
:101BDB009001BCF0A3F09001B9F09001B9E0F9C30A
:101BEB0094064003021C83A3E0FF14F074742FF5DA
:101BFB0082E43400F583E0FF9001BBE08FF0A4FD9D
:101C0B00A3E07E002DFFEE35F0FEE9FDC374059DCC
:101C1B00FDE49400FC1225F3E07A002FFFEA3E90DE
:101C2B0001BCF0A3EFF09001BCA3E0FF1225F3EF92
:101C3B00F0E904FDEDC3940650359001BCE0FF7E46
:101C4B0000EEF0A3EFF06027EDFFC374059FFFE4F8
:101C5B009400FE1225FEE0FB9001BCE48BF0120217
:101C6B00559001BCA3E0FC1225FEECF00D80C59055
:101C7B0001B9E004F0021BE59001BAE02406F00282
:101C8B001B849001AEE0FF7B017A0179B39001C216
:061C9B007406F0022A07A6
:03268E00CBEFCBC4
:10269100C3EC648094805008ED2410FDEC340EFCF2
:1026A100CEECCECFEDCF7C3F7DFF1201B87C0E7D0D
:1026B1001012021FEE543FFE3395E0FDFC9001AE77
:1026C100120413CFEBCF0BEFC0E09001AE1203FB6E
:1026D10078081203D4CDEFCDD0E0FF122D40CFEB1F
:1026E100CFEFC0E09001AE1203FBE4CDEFCDD0E01F
:0426F100FF022D4077
:0320C500CAEFCA95
:1020C800E4FB9001AE740FF0A374FFF0EA642160A2
:1020D80003022159C312260950097B2074962DFD4D
:1020E800E43CFCC3EC64809480405EED942CEC648A
:1020F800809481400CEB4402FB74D42DFD74FE3CAB
:10210800FCC3ED94C8EC648094804009EB4404FB64
:102118007438122614C3ED9464EC648094804009EA
:10212800EB4408FB749C122614C3ED9432EC6480D3
:1021380094804009EB4410FB74CE12261412261B1F
:1021480040047C007D311225C8CFEBCF122CEF80E4
:1021580016C3E41226095003E4FCFD12261B4004B2
:102168007C007D311225C8C9EAC90ACFE9CFEFC082
:10217800E09001AEE0FEEEFDD0E0FF122D40CFEA88
:0A218800CF9001AEA3E0FD022D4050
:0B279E009001AEEFF0CBEDCBCAECCA0F
:1027A900CFEBCFCEEACEE4FCFD7BFF7A0FF9F8122E
:1027B90002861225E7E47BE87A03F9F8120311127D
:1027C90025E7EE6408FACBEFCB9001AEE0FF04F009
:1027D900EAFD122D409001AEE0FFCDEBCD022D4078
:052DA400E4FF022CEF2A
:102751009001AE120413122B8D7C007D0A1201CA66
:10276100CBEFCBCAEECAE4F9F81225C2EF24FFFF82
:10277100EE34FFFEED34FFFDEC34FFFC1202861255
:1027810025BCCDEF7F1C1225ADCDEF7F1B1225ADF2
:0D279100EF540FFFE4CDEFCD7F1A022D4075
:1017C3004261636B6C69676874004F6E004F6666B5
:1017D300004368616E6E656C2051005265666572E8
:1017E300656E63650053696E6500436F6D7061726A
:1017F30061746F720053696E632066696C746572FD
:1018030000506F776572646F776E206D6F6465004B
:1018130053696E7573206F757470757400506861C9
:101823007365206D6F64756C6174696F6E004672C9
:1018330065712E206D6F64756C6174696F6E0046FF
:101843007265712E206D6F642E202B207377656572
:101853007000547269616E67756C6172207377658D
:10186300657000536C656570206D6F646500556E1F
:101873007265636F676E697A6564206D6F64650076
:101883004D61696E206672657175656E637900419D
:101893006C742E206672657175656E6379004D6197
:1018A300696E20706861736500416C742E207068E6
:1018B30061736500416D706C6974756465204900DE
:1018C30044757479206379636C65205100526566B1
:1018D3006572656E6365205100416D706C69747546
:1018E30064652051005377656570207265736F6C72
:1018F3007574696F6E0053776565702066726571E4
:101903002E20737465700057726F6E67207061725A
:10191300616D6574657200496E707574206C6F63D8
:101923006B656420627920686F7374004D6F646522
:1019330020467265712E20416D702E20202E2E2E92
:101943000053797374656D204D656E7500504C4C72
:1019530020427970617373656400504C4C206D753F
:101963006C742E202564780051756172747A202579
:101973003364204D487A003D0050726576204E65F1
:0E19830078742043687E67652045786974009B
:101A6D004100DC0041013E004800BC0101010101C3
:101A7D00010101460145313D33F3F3004400C80037
:101A8D000F42404400CC000F42404400D8000003F8
:101A9D00E84200D6000A4400B807270E004200C4F1
:101AAD00FDA84200C6FDA84200D000004200D203AE
:101ABD00844200D403E841013F014101410141014C
:101ACD0043004101440041014C0141014B004101E2
:101ADD0037014101400042013C0014605A00DD0114
:101AED000137FF17C3FF17CDFF17D000000001010D
:101AFD004CFF17D4FF17DEFF17E8FF17D001014188
:101B0D00FF17EDFF17CDFF17D0000000010143FFB8
:101B1D0017F8FF17CDFF17D0000000010144FF1883
:101B2D0004FF17CDFF17D0000000000000000000DB
:101B3D00000000000000000000440138144F012097
:1024AA009000B81203FB90015E120413900162744B
:1024BA0009F0E4A3F0741BA3F07401A3F090013EA9
:1024CA00E024BCF9E43400FA7B019001660204734B
:1024DA00EF75F00FA424DDF582E43400F5830204DD
:1024EA0053E0FEA3E0FFEE3395E0FDFCEC22740618
:1024FA00900162F0A37401F0A3221203FB9001AFD2
:10250A0002041375F00FA424E9F582E43400F5837C
:10251A000204539000D6E0FEA3E0FFE4FCFD229003
:09252A0001407401F090013A2215
:102A70007B017A017954E4FDFC122BB0900157E000
:102A8000900139F0900155A3E0FF90013CE4F0A3E0
:0F2A9000EFF07B017A0079B87D487C00022BB013
:1022E300E4FF900141E070037410FF90014CE0FEA5
:1022F300B40204EF4404FF900144E06004EF441788
:10230300FF900138EFF0E4900140F09000DCE0141E
:10231300601814601D14602214602714602C2405B7
:10232300702E90013A7401F0802690013A7409F0FE
:10233300801E90013A7403F080161225297405F06B
:10234300800E1225297425F080069001387417F049
:10235300EEB4010790013AE04410F090013B742081
:10236300F0900143E0700790013BE04440F07B01B3
:102373007A0179389001C27404F07F1D122A079004
:072383000137E0FF022C6DA1
:10219200900140E0FF601460229000CC1203FB909B
:1021A20000C8120407C31203BE50109000C81225C3
:1021B200047F04121B569000CC800E9000CC122596
:1021C200047F04121B569000C81225047F0A121BBA
:1021D2005612251D1227519000D81225047F101285
:1021E2001B569000D0E0FCA3E0FDE4FF12268E9087
:1021F20000D2E0FCA3E0FD7F0212268E90013FE0B8
:102202006006900144E06003022DA49000C4E0FC4B
:10221200A3E0FD7F211220C590014CE0B4010D9096
:1022220000D4E0FCA3E0FD7F2602279E9000C6E0DA
:0A223200FCA3E0FD7F231220C5226B
:101DC5007F01122ACD9000DCE014601814601D1408
:101DD500602214602714602C240570307BFF7A186C
:101DE5007913802E7BFF7A18792080267BFF7A185D
:101DF5007931801E7BFF7A18794280167BFF7A182D
:101E05007955800E7BFF7A18796680067BFF7A18F4
:101E15007971900156120473900156120453E4FF30
:101E2500122A9F90013EE012047C1E4B001E5301B6
:101E35001E5B021E63031E6B041E73051E96061EA3
:101E45009E0700001EA67BFF7A18798380397BFFE9
:101E55007A18799280317BFF7A1879A180297BFFE6
:101E65007A1879AC80217BFF7A1879B7803990018F
:101E75004CE0B40114900141E07BFF60067A1879CB
:101E8500C380047A1879D0801E7BFF7A1879DC80AC
:101E9500167BFF7A1879E8800E7BFF7A1879F9802E
:101EA500067BFF7A19790A9001561204737FC012D6
:101EB5002ACD7F7E122D689001561204537F411260
:101EC5002A9F90014BE07BFF60067A19791A8004FE
:091ED5007A19792F7F54122A9F1B
:011EDE0022E1
:1028340090013EE0FFFE7401C8EFC8088002C33374
:10284400D8FCFF7DFF90013FE070027DCF90014CEA
:10285400E0B40204ED54DFFDEEC3940850170EEF0C
:1028640025E0FF9000DCE02445F582E43401F583A3
:09287400E05F5D60E3EE5407FF34
:01287D002238
:1012A400E4900154F0A304F0122533900154EFF0BC
:1012B40024BE604314604214605424F5607324E235
:1012C4006056242C70709000DCE0FFB4050B900194
:1012D40042E09000DCF0E48018EFC394044007E49B
:1012E4009000DCF080069000DCE004F0E490013E25
:1012F400F0900144F0803F800E90013FE060089040
:10130400013E7404F0802FE490013EF080281228FE
:101314003490013EEFF0801E1215C4900144E06049
:10132400159000DCE0900142F09000DC7405F08040
:1013340005E4900154F090014BE06022121DC57F3A
:101344004C122D4E90014BE0600F12253390015446
:10135400EFF060F0121DC580EB7F55122D4E900109
:1013640054E07004A3E06008121DC5E4900155F038
:101374001222E312219290013EE012047C139D009C
:1013840013B50113D102141603145C0414A4051537
:101394004006158907000012AC90015A12041F0080
:1013A4000000001224AA9000C81215BD9000C88045
:1013B4001690015A12041F000000001224AA900083
:1013C400CC1215BD9000CC1204130212AC9000D0C4
:1013D4001224EBC0E0EDC0E0EEC0E0EFC0E090010D
:1013E4005A12041FFFFFF8F890015E12041F000058
:1013F40007081224F8741EF074051224C5D0E0FF07
:10140400D0E0FED0E0FDD0E0FC1204BB9000D0029E
:1014140015819000D21224EBC0E0EDC0E0EEC0E0F4
:10142400EFC0E090015A12041FFFFFF8F890015E2C
:1014340012041F000007081224F8741EF0A3740598
:101444001224C6D0E0FFD0E0FED0E0FDD0E0FC12D4
:1014540004BB9000D20215819000C41224EBC0E0BA
:10146400EDC0E0EEC0E0EFC0E090015A12041FFFAF
:10147400FFFD4590015E12041F00000096740512E2
:1014840024FA741FF0A374041224C6D0E0FFD0E041
:10149400FED0E0FDD0E0FC1204BB9000C402158134
:1014A40090014CE014704B9000D41224EBC0E0ED9A
:1014B400C0E0EEC0E0EFC0E090015A12041F00004B
:1014C400000090015E12041F000003E890016274A2
:1014D400051224FD741FF0A374021224C6D0E0FF89
:1014E400D0E0FED0E0FDD0E0FC1204BB9000D402BA
:1014F40015819000C61224EBC0E0EDC0E0EEC0E020
:10150400EFC0E090015A12041FFFFFFFCF90015E6D
:1015140012041F0000000090016274051224FD747F
:101524001FF0A374041224C6D0E0FFD0E0FED0E084
:10153400FDD0E0FC1204BB9000C6804112251DECD6
:10154400C0E0EDC0E0EEC0E0EFC0E090015A12044C
:101554001F0000000190015E12041F000080E812C9
:1015640024F8741FF0A374061224C6D0E0FFD0E060
:10157400FED0E0FDD0E0FC1204BB9000D6EEF0A358
:10158400EFF00212AC90015A12041F000000019007
:10159400015E12041F000186A09001627406F0E44B
:1015A400A3F0741E1224C19000D81203FB1204BBD2
:0915B4009000D81204130212ACDD
:0715BD001203FB1204BB2224
:102B8D00900139E0FD30E50990013CE0FEA3E0FF46
:102B9D0022ED541FFF7E0090013CE0FCA3E0FD12EE
:032BAD0001B8224A
:1015C400E4900156F0A304F0900157E07003021672
:1015D400BB7F01122ACD7BFF7A197944E4FF122ADA
:1015E4009F7F93122ACD900156E02431FF122D687B
:1015F400900156E064057045900139E07BFF30E5C9
:10160400067A19795080157A19795D9000031204CD
:1016140073900139E0541FFFE41217AC7F40122A83
:101624009F7BFF7A19796B90000312047390013C3D
:10163400E0FFA3E0CF1217AC7F140216AD90015661
:10164400E075F00FA424E0F582E43400F58312047D
:10165400537F40122A9F7BFF7A19797A7F14122ACA
:101664009F900156E0FF1224DB12011C24FE601837
:10167400047020EF75F00FA424E3F582E43400F540
:10168400831204537F168021900156E012250D7FAA
:10169400168016900156E075F00FA424E6F582E456
:1016A4003400F5831204537F16122A9F7BFF7A19A4
:1016B400797C7F54122A9F122533900157EFF01240
:1016C400047C17AB2117022B16EE2D17AB3C17AB7E
:1016D4003E16EE4117024217164317AB4417AB45AB
:1016E40017AB5217AB6D00001759900156E0600517
:1016F40014F00215CC9001567405F00215CC90013B
:1017040056E004F0E0D3940550030215CCE4F00253
:1017140015CC900156E0FF640570030215CC122429
:10172400DA7401120162900156E0FF12250DE94AB4
:10173400700A1224DA12011C54018010900156E040
:101744001224DB12011CD394024004E4120184121B
:1017540022E30215CC122D10900158EEF0A3EFF005
:101764004E70030215CC122BD3D3900159E0940090
:10177400900158E0648094804014900156E09405F0
:101784004004E4F08018900156E004F080109001C9
:1017940056E0600414F080069001567405F0900140
:0717A400577401F00215CC9F
:1017AB0022900006F0A3EFF07B017A01795A120C1C
:0817BB007A7B017A01795A22C0
:081B4D004101EE014101EF002E
:1029D0007A0179A37B019001A2E09001B2227B01F0
:1029E0007A0179A49001A8E0FCA3E0FD22E0FF04B5
:1029F000F074B32FF582E43401F583229001B1E045
:072A0000FF9001B8E09F22E6
:0B2625009001AE1204739001B1EDF0C3
:10263000E49001B8F0D31229FC50277FF47E0112F8
:102640002C35EF601AE49001EFF0AD999001B2E003
:10265000CFEDCF6DF09001B81229EDEDF080D67F6F
:1026600000229001B2E060037F0022E49001B8F004
:10267000C31229FC50151229EDE0FF9001AEE4755C
:0D268000F00112045CEF12018480E57F017F
:01268D00222A
:0E2D4E009001EEE060FA8F99E49001EEF02221
:100F79009001A2E599F0E49001EFF07F52122D4E15
:100F89009001A2E0FF12047C0FD4000FDD010FE9EC
:100F9900020FF2030FFB04100405100D06101607CB
:100FA900102108103009103F0A104E0B105D0C106B
:100FB9006C0D107A0F109010109E1110B71210C5F9
:100FC9002010D130116E31000011AA9001A17401D5
:100FD900F00211AF7B017A0079C89001B2EF80412C
:100FE9007A0079CC1229D480387B017A0079C4023D
:100FF90010BD7B017A0079C60210BD7B017A0079A8
:10100900D00210BD7B017A0079D20210BD7B017A32
:101019000079D61229D680097B017A0079D812295C
:10102900D6F07D040210CB7B017A01793F1229D6D3
:10103900F07D010210CB7B017A0179411229D6F0AA
:101049007D010210CB7B017A0179431229D6F07D0B
:10105900010210CB7B017A0179441229D6F07D0176
:101069000210CB7B017A01794C1229D6F07D0180DF
:10107900519000DCE0900142F07B017A0079DC12AA
:1010890029D6F07D01803B7B017A0179371229D677
:10109900F07D01802D1229D0F07D0112129B700381
:1010A9000211AF9001A3E0FF122BF50211AF7B01F2
:1010B9007A0079D41229D6F07D0280061229D0F05F
:1010C9007D0112129B0211AFE49001A8F0A3F07BFD
:1010D900017A0179A41229D6F07D041226259001FE
:1010E900A1EFF0FB9001A4E0FFE4FCFDFE9001AA52
:1010F900120413EB6012121248E49001A3F01212C9
:101109000C600512124880030212069001A3E00444
:10111900F0E0C3941140E712120C600D1229DE129F
:1011290028C57F21122D4E800302120612125F601C
:101139000D1229DE1228C57F21122D4E80030212BD
:101149000612125F60061229DE1228C59001A1E07D
:1011590060109001AA1203FBEC4D4E4F70047F21E1
:10116900803A0212067B017A0179A81229D6F07D0C
:10117900021226259001A1EFF01229DE122BB09060
:1011890001A4E0FF122D4E9001A5E0FF122D4E9013
:1011990001A6E0FF122D4E9001A7E0FF122D4E800F
:1011A90005E49001A1F09001A1E060517F21122D89
:1011B9004E7F45122D849001A2E0FE64207029A380
:1011C900E0FF90014BE05F60057F4C122D4E9001CE
:1011D900A3E0FF90014BE04F70057F55122D4E9013
:1011E90001A3E090014BF022EED39430501490010A
:1011F900A2E0D3940840031222E30221927F3F1216
:021209002D4E68
:10120B00229001A8E475F0041202557B017A017952
:10121B00A4E49001B2F07D041226259001A1EFF019
:10122B009001AA1204079001A4E0FFE4FCFDFE125A
:10123B0003A39001AA1204139001A1E0227B017A6F
:10124B000179A49001A8E0FCA3E0FD1228C57F2141
:10125B00122D4E229001A8E475F0041202557B0169
:10126B007A0179A4E49001B2F07D04122625900155
:10127B00A1EFF09001AA1204079001A4E0FFE4FC97
:10128B00FDFE1203A39001AA1204139001A1E02208
:09129B001226259001A1EFF022BA
:062B4600CEECCECFEDCF76
:102B4C00CDEFCDCCEECCED7802CEC313CE13D8F9AD
:0E2B5C00F5C6EC1313543FF5C7ED5403FF22EA
:1028C5009001AE7404F0122B4612011CF5BC900069
:1028D50001120135F5BD900002120135F5BE9000DB
:1028E50003120135F5BF75B90575B90275B904AFA0
:1028F500B9EF60089001AEE014F070EAEF70047F64
:052905000180027F00CB
:01290A0022AA
:102BB000122B4675B901E5BC120184900001E5BDF8
:102BC000120196900002E5BE120196900003E5BF47
:032BD00002019669
:1027E900E4FFFEFDFC900154F0F9F5C7FB8BC675BB
:1027F900B901E5BC6FFFE5BD6EFEE5BE6DFDE5BF48
:102809006CFCEBB41108A9BE900154E5BFF00BEBC9
:10281900B415DAE964557010900154E0B4AA09EFCF
:0A2829004E4D4C70037F01227F002A
:012833002282
:10239C00022992E493A3F8E493A34003F68001F29C
:1023AC0008DFF48029E493A3F85407240CC8C33342
:1023BC00C4540F4420C8834004F456800146F6DF11
:1023CC00E4800B0102040810204080901991E47EF7
:1023DC00019360BCA3FF543F30E509541FFEE49306
:1023EC00A360010ECF54C025E060A840B8E493A3CD
:1023FC00FAE493A3F8E493A3C8C582C8CAC583CAF8
:10240C00F0A3C8C582C8CAC583CADFE9DEE780BEAF
:011B5500008F
:10002600E709F608DFFA8046E709F208DFFA803EBC
:1000360088828C83E709F0A3DFFA8032E309F608A9
:10004600DFFA8078E309F208DFFA807088828C8311
:10005600E309F0A3DFFA806489828A83E0A3F608C5
:10006600DFFA805889828A83E0A3F208DFFA804C9F
:1000760080D280FA80C680D4806980F28033801076
:1000860080A680EA809A80A880DA80E280CA8033DF
:1000960089828A83ECFAE493A3C8C582C8CCC58357
:1000A600CCF0A3C8C582C8CCC583CCDFE9DEE78027
:1000B6000D89828A83E493A3F608DFF9ECFAA9F0A6
:1000C600EDFB2289828A83ECFAE0A3C8C582C8CCFC
:1000D600C583CCF0A3C8C582C8CCC583CCDFEADE15
:1000E600E880DB89828A83E493A3F208DFF980CC77
:1000F60088F0EF60010E4E60C388F0ED2402B40470
:100106000050B9F582EB2402B4040050AF23234516
:06011600822390007673C5
:10011C00BB010689828A83E0225002E722BBFE02E1
:09012C00E32289828A83E4932214
:10013500BB010CE58229F582E5833AF583E022507F
:1001450006E92582F8E622BBFE06E92582F8E222C9
:0D015500E58229F582E5833AF583E49322E3
:10016200BB010989828A83F8E028F022500327F72D
:1001720022BBFE05F8E328F3228A838982F8E493FE
:02018200282231
:10018400BB010689828A83F0225002F722BBFE015A
:02019400F32254
:10019600F8BB010DE58229F582E5833AF583E8F09F
:1001A600225006E92582C8F622BBFE05E92582C84B
:0201B600F22233
:1001B800EF8DF0A4A8F0CF8CF0A428CE8DF0A42E5B
:0201C800FE2215
:1001CA00BC000BBE0029EF8DF084FFADF022E4CC19
:1001DA00F875F008EF2FFFEE33FEEC33FCEE9DECE2
:1001EA00984005FCEE9DFE0FD5F0E9E4CEFD22ED28
:1001FA00F8F5F0EE8420D21CFEADF075F008EF2F72
:10020A00FFED33FD4007985006D5F0F222C398FD62
:05021A000FD5F0EA22FF
:10021F00C2D5EC30E709B2D5E4C39DFDE49CFCEEFA
:10022F0030E715B2D5E4C39FFFE49EFE1201CAC3A7
:10023F00E49DFDE49CFC80031201CA30D507C3E4A2
:06024F009FFFE49EFE2269
:10025500C5F0F8A3E028F0C5F0F8E5821582700234
:060265001583E038F022D1
:0D026B00EF2BFFEE3AFEED39FDEC38FC22E2
:0E027800C3EF9BFFEE9AFEED99FDEC98FC2281
:10028600E88FF0A4CC8BF0A42CFCE98EF0A42CFC17
:100296008AF0EDA42CFCEA8EF0A4CDA8F08BF0A495
:1002A6002DCC3825F0FDE98FF0A42CCD35F0FCEBF4
:1002B6008EF0A4FEA9F0EB8FF0A4CFC5F02ECD39B9
:0F02C600FEE43CFCEAA42DCE35F0FDE43CFC2226
:1002D50075F008758200EF2FFFEE33FECD33CDCCE0
:1002E50033CCC58233C5829BED9AEC99E582984063
:1002F5000CF582EE9BFEED9AFDEC99FC0FD5F0D640
:10030500E4CEFBE4CDFAE4CCF9A88222B800C1B969
:100315000059BA002DEC8BF084CFCECDFCE5F0CBA7
:10032500F97818EF2FFFEE33FEED33FDEC33FCEBE0
:1003350033FB10D703994004EB99FB0FD8E5E4F99B
:10034500FA227818EF2FFFEE33FEED33FDEC33FC88
:10035500C933C910D7059BE99A4007EC9BFCE99A7C
:10036500F90FD8E0E4C9FAE4CCFB2275F010EF2FC1
:10037500FFEE33FEED33FDCC33CCC833C810D707C1
:100385009BEC9AE899400AED9BFDEC9AFCE899F8FC
:0E0395000FD5F0DAE4CDFBE4CCFAE4C8F9228F
:10290B00C2D5E830E70FB2D5E4C39BFBE49AFAE4F7
:10291B0099F9E498F8EC30E717B2D5122941120374
:10292B0011E4C39BFBE49AFAE499F9E498F8800369
:10293B0012031130D50DE4C39FFFE49EFEE49DFD11
:04294B00E49CFC22EA
:0D03A300EF6BFFEE6AFEED69FDEC68FC22D9
:0E03B000C3E49FFFE49EFEE49DFDE49CFC225E
:1003BE00EB9FF5F0EA9E42F0E99D42F0EC6480C8B6
:0603CE0064809845F02256
:1003D400E8600FECC313FCED13FDEE13FEEF13FF07
:0303E400D8F1222B
:1003E700E86010ECA2E713FCED13FDEE13FEEF132C
:0403F700FFD8F02219
:0C03FB00E0FCA3E0FDA3E0FEA3E0FF2275
:0C040700E0F8A3E0F9A3E0FAA3E0FB2278
:0C041300ECF0A3EDF0A3EEF0A3EFF0225C
:10041F00A8828583F0D083D0821204391204391256
:10042F000439120439C082C08322E493A3C583C563
:10043F00F0C583C8C582C8F0A3C583C5F0C583C8FE
:04044F00C582C82278
:09045300E0FBA3E0FAA3E0F922AA
:10045C00F8E0FBA3A3E0F925F0F0E5821582700229
:07046C001583E0FA38F022CD
:09047300EBF0A3EAF0A3E9F0228A
:10047C00D083D082F8E4937012740193700DA3A30F
:10048C0093F8740193C0E0E8C0E0227402936860B2
:06049C00EFA3A3A380DF23
:100C1E00E5082403F8E2050822780030070278037D
:100C2E00E475F0011204A202011C2000EB7F2ED20B
:100C3E00008018EF540F2490D43440D4FF30040BAE
:100C4E00EF24BFB41A0050032461FFE509600215BA
:100C5E0009050CE50C7002050B30070D7800E475E4
:100C6E00F0011204A2EF020184022B1F7403D207BB
:100C7E008003E4C207F50878001204B2E4F509F522
:100C8E000BF50CE50960077F20120C5980F5750AEB
:100C9E00FFC201C200C202C203C205C206C20812CE
:100CAE000C27FF700D3007057F00120C6AAF0CAEDB
:100CBE000B22B4255FC2D5C204120C27FF24D0B478
:100CCE000A00501A75F00A780930D50508B6FF01EA
:100CDE0006C6A426F620D5047002D20380D924CFEE
:100CEE00B41A00EF5004C2E5D204020E69D201809C
:100CFE00C6D20080C0D20280BCD2D580BAD20580C6
:100D0E00B47F20120C592002077401B5090040F17E
:100D1E00120C1EFF120C59020C91D208D2068095AD
:100D2E00120C1EFB120C1EFA120C1EF94A4B700608
:100D3E00793A7A0F7BFF20022EE509602A7E008E1B
:100D4E008275830012013560060EEE650A70F0C2E0
:100D5E00D5EBC0E0EAC0E0E9C0E0EE120EB0D0E0A4
:100D6E00F9D0E0FAD0E0FB12011CFF60AAEBC0E064
:100D7E00EAC0E0E9C0E0120C59D0E02401F9D0E05D
:100D8E003400FAD0E0FBE50A0460DCD50AD980878E
:100D9E007BFF7A0E79ACD202809C791080027908A2
:100DAE00C206C2088008D2D5790A8004790AC2D553
:100DBE00E50A047002F50AE4FAFDFEFF120C1EFCB1
:100DCE007B08200113120C1EFD7B1030000A120C42
:100DDE001EFE120C1EFF7B20EC3382D592D55013D3
:100DEE00C3E43000069FFFE49EFEE42001039DFD58
:100DFE00E49CFCE4CBF8C201EC700CCFCECDCCE879
:100E0E0024F8F870F38017C3EF33FFEE33FEED33A3
:100E1E00FDEC33FCEB33FB994002FB0FD8E9EB30D2
:100E2E000105F8D0E0C448B201C0E00AEC4D4E4FC7
:100E3E0078207B0070C2EAB50A0040BCC0E0120EFA
:100E4E00B2D0F0D0E0200104C4C0E0C4B201C0F0C2
:100E5E00120C42D0F0D5F0EB020C9112047C0D2E48
:100E6E00530DA8580CFF4C0CFB420DAC4F0DB44467
:100E7E000DB4490D14430DBA550D9E460D9E450DEC
:010E8E009EC5
:100E8F00470F5A500D032D0D072E0D2A2B0D0B2337
:100E9F000D28200F432A0CC34800000D223F3F3F6F
:100EAF0000790AA2D5200314300509B910020404F1
:100EBF00B9080104A2D5200602500104200268924D
:100ECF0002B509005034C0E07F203003197F30A2F3
:100EDF000272067205500F120F09C202C206C20536
:100EEF00C2087F30800F300503E9C0E0120C593083
:100EFF000503D0E0F9D0E0B509CC3005177F30B944
:100F0F00100C120C597F583004077F788003B908F2
:100F1F0003120C593002057F2D020C597F20200837
:100F2F00F87F2B2006F322920280CF286E756C6C0F
:100F3F002900D201120C1E3001F8C201780930D5F8
:100F4F000108F6020CC32D50434958120C1E2403FE
:100F5F00B405004001E4900F5593120C4A743A12F5
:0A0F6F000C4AD203750904020DA814
:1004A200FAE2FB0808E2F925F0F218E2CA3AF2226F
:0904B200EBF208EAF208E9F2227B
:102B1F00EFB40A07740D122B2A740A309811A89972
:102B2F00B8130CC2983098FDA899C298B811F63016
:072B3F0099FDC299F59922EE
:00000001FF
